:100000000C945F000C9489000C9489000C94890076
:100010000C9489000C9489000C9489000C9489003C
:100020000C9489000C9489000C9489000C9489002C
:100030000C9489000C9489000C9489000C9489001C
:100040000C9489000C9489000C9489000C9489000C
:100050000C9489000C9489000C9489000C948900FC
:100060000C9489000C9489000C9489000C948900EC
:100070000C9489000C9489000C9489000C948900DC
:100080000C9489000C9489000C948900F800FB0002
:10009000FE00EF000101040107010A010D0110013A
:1000A000F5001301AA05A705A4056105A1059E0594
:1000B0009B059805950592058F05AD05B0051124A2
:1000C0001FBECFEFD0E4DEBFCDBF11E0A0E0B1E0B6
:1000D000E4ECFBE000E00BBF02C007900D92A232FF
:1000E000B107D9F721E0A2E2B1E001C01D92A4332B
:1000F000B207E1F710E0CFE5D0E004C02197FE01A0
:100100000E94D705CE35D107C9F70E944A050C9445
:10011000E0050C94000083E391E00E94170160E089
:1001200080E391E00E945A016FEF80E391E00E942A
:100130007B0160E08DE291E00E945A016FEF8DE259
:1001400091E00E947B016FEF8AE291E00E947B01C7
:1001500083E291E00E94520282E291E00E944A030F
:10016000789484B7877F84BF109260000FB6F894AC
:10017000A895809160008861809360001092600073
:100180000FBE0895CF930FB6F894A89580916000A4
:10019000886180936000109260000FBE6FEF8DE267
:1001A00091E00E949C0182E291E00E940E04C82F1F
:1001B00060E08DE291E00E949C0199E288E10FB637
:1001C000F894A895809360000FBE90936000A89566
:1001D0008C2F90E0FC013197EC30F10510F0CF91BD
:1001E0000895EA5BFF4F0C94D705CF910C94C60499
:1001F000CF910C942604CF910C943704CF910C949A
:100200005B04CF910C946804CF910C947B04CF9144
:100210000C948E04CF910C949704CF910C94A0046D
:10022000CF910C94B304CF910C94D404089584B16D
:10023000806B84B926988AB18C618AB980E58CBDBF
:1002400081E08DBD8BB1837E8BB95A9A5B9A5C9AA3
:1002500008958BB1837E8BB98BB160FD10C090E0A7
:10026000892B8BB98BB161FD10C090E0892B8BB9C4
:100270008BB162FD10C090E0892B8BB9089594E09A
:10028000892B8BB98BB161FFF0CF98E0892B8BB9AB
:100290008BB162FFF0CF90E1892B8BB908956EBDD1
:1002A0000DB407FEFDCF8EB50895FC017183608308
:1002B000428308951F93CF93DF93EC01162F6A8139
:1002C000888199810E94290160E4888199810E9436
:1002D0004F0160E0888199810E944F01612F8881E0
:1002E00099810E944F0167E088819981DF91CF91C8
:1002F0001F910C9429011F93CF93DF93EC01162FCC
:100300006A81888199810E94290160E488819981AC
:100310000E944F0161E0888199810E944F01612F05
:10032000888199810E944F0167E088819981DF91DE
:10033000CF911F910C9429011F93CF93DF93EC0170
:10034000162F6A81888199810E94290160E4888141
:1003500099810E944F0162E1888199810E944F0139
:10036000612F888199810E944F0167E0888199817E
:10037000DF91CF911F910C9429011F93CF93DF93AD
:10038000EC01162F6A81888199810E94290160E41D
:10039000888199810E944F0163E1888199810E943F
:1003A0004F01612F888199810E944F0167E0888108
:1003B0009981DF91CF911F910C9429011F93CF93C5
:1003C000DF93EC016A81888199810E94290161E4AF
:1003D000888199810E944F0162E1888199810E9400
:1003E0004F0160E0888199810E944F01182F67E0DA
:1003F000888199810E942901812FDF91CF911F91DE
:1004000008951F93CF93DF93EC016A8188819981CE
:100410000E94290161E4888199810E944F0163E172
:10042000888199810E944F0160E0888199810E94B2
:100430004F01182F67E0888199810E942901812F3F
:10044000DF91CF911F910895FC01718360834283F6
:1004500008950F931F93CF93DF93EC018B016A8173
:10046000888199810E942901B8010024660F771FB5
:10047000001C660F771F001C672F702D88819981E3
:100480000E944F01602F660F660F888199810E943C
:100490004F0167E088819981DF91CF911F910F9182
:1004A0000C94290110927C0087E880937A000895CB
:1004B00080917C00807E682B60937C0080917A0024
:1004C000806480937A0083EA91E00197F1F700C09D
:1004D000000080917A0086FDFCCF80917800909199
:1004E000790008950F931F93CF93DF9361E080E32A
:1004F00091E00E949C01C1E0D0E001E010E02FEF0C
:1005000084E39CE0215080409040E1F700C000006F
:10051000B8010C2E01C0660F0A94EAF780E391E05F
:100520000E949C012196C930D10549F7DF91CF91F6
:100530001F910F9108950F931F93CF93DF9361E065
:100540008DE291E00E949C01C1E0D0E001E010E06A
:100550002FEF84E39CE0215080409040E1F700C001
:100560000000B8010C2E01C0660F0A94EAF78DE274
:1005700091E00E949C012196C930D10549F7DF9195
:10058000CF911F910F910895CF93DF93C0E0D0E0FA
:10059000BE0187E291E00E94290287E893E101977A
:1005A000F1F700C000002196C11594E0D90781F74A
:1005B0002FE78AE196E0215080409040E1F700C0AB
:1005C000000060E070E087E291E0DF91CF910C9451
:1005D0002902CF93DF93C0E0D0E0BE0184E291E036
:1005E0000E94290287E893E10197F1F700C000001B
:1005F0002196C11594E0D90781F72FE78AE196E0AB
:10060000215080409040E1F700C0000060E070E0C1
:1006100084E291E0DF91CF910C9429020FB6F89417
:10062000A8958091600088618093600010926000BE
:100630000FBE60E083E291E00E945802BC0187E2B5
:1006400091E00E94290261E083E291E00E94580259
:10065000BC0184E291E00E94290280E391E00E94C3
:100660000102682F80E391E00E949C018AE291E000
:100670000E940102682F8DE291E00E949C01D9CF77
:100680000E9472020E949B020E94C4020E94E90220
:100690000E940E0382E08093C00088E18093C10035
:1006A00086E08093C2001092C50080E48093C4006D
:1006B00008958091C00085FFFCCF6093C6008091B3
:1006C000C00086FFFCCF08958091C00085FFFCCF5D
:1006D0006093C6008091C00085FFFCCF7093C60078
:1006E0008091C00086FFFCCF87E893E10197F1F786
:1006F00000C0000008958091C00085FFFCCF4093AA
:10070000C6008091C00086FFFCCFFB019B01240F37
:10071000311DE217F30761F091918091C00085FFD0
:10072000FCCF9093C6008091C00086FFFCCFF1CF34
:1007300008958091C00085FFFCCF4093C600809152
:10074000C00086FFFCCF5FEF540F442309F464C060
:10075000FB0120E041E9DF0190818091C00085FF2D
:10076000FCCF9093C6008091C00086FFFCCF3196ED
:100770009C91822F892780FD842790E0959587950D
:10078000282F80FF02C0242F2827822F90E09595E4
:100790008795282F80FF02C0242F282730E0359529
:1007A0002795822F20FF02C0842F822790E0959505
:1007B0008795282F80FF02C0242F282730E0359509
:1007C0002795822F20FF02C0842F822790E09595E5
:1007D0008795282F80FF02C0242F282730E03595E9
:1007E0002795822F20FF02C0842F8227282F26954D
:1007F000515008F0B0CF8091C00085FFFCCF20930E
:10080000C6008091C00086FFFCCF8091C00087FFAA
:10081000FCCF8091C600089520E0EDCF8091C0000C
:1008200087FFFCCF8091C60008958091C00087FFAC
:10083000FCCF2091C60030E09091C00097FFFCCF24
:100840008091C600A901582BCA010895CF9382E276
:1008500091E00E940E04C82F6FEF82E291E00E94A7
:1008600059036C2F82E291E0CF910C94590363E01D
:1008700082E291E00E9459034CE066E171E082E27D
:1008800091E00E947B0349E06DE071E082E291E03B
:100890000E947B034CE061E071E082E291E00E9403
:1008A0007B0380910001811101C008956FEF82E206
:1008B00091E00C94590382E291E00E941504BC017E
:1008C000660F771F680F791F82E291E00C94640332
:1008D00082E291E00E940E04682F80E391E00E9482
:1008E0009C0180910001811101C008956FEF82E2A7
:1008F00091E00C94590382E291E00E940E04682F6B
:100900008DE291E00E949C0180910001811101C063
:1009100008956FEF82E291E00C94590380E391E037
:100920000E940102682F82E291E00C9459038DE24B
:1009300091E00E940102682F82E291E00C94590339
:1009400082E291E00E941504BC0187E291E00E94DE
:10095000290280910001811101C008956FEF82E2A8
:1009600091E00C94590382E291E00E941504BC01CD
:1009700084E291E00E94290280910001811101C06E
:1009800008956FEF82E291E00C94590382E291E0C6
:100990000E940E04682F83E291E00E945802BC017D
:1009A00082E291E00C9464038F929F92AF92BF9287
:1009B000CF92DF92EF92FF920F931F93CF93DF932B
:1009C00000D000D0CDB7DEB782E291E00E940E04E5
:1009D000B82E82E291E00E940E04A82E82E291E0FD
:1009E0000E9415048C0182E291E00E9415047C01B2
:1009F00082E291E00E9415044C016FEF82E291E0E7
:100A00000E945903E89C6001E99CD00CF89CD00C32
:100A100011240C151D05C4F5B80187E291E00E9470
:100A20002902A8956B2D83E291E00E9458029A83D7
:100A300089836A2D83E291E00E9458029C838B8314
:100A400002C08F3FE1F0A89544E0BE016F5F7F4F89
:100A500082E291E00E9499038111F3CF0F900F90F1
:100A60000F900F90DF91CF911F910F91FF90EF901A
:100A7000DF90CF90BF90AF909F908F9008950E0D14
:100A80001F1D0C151D0544F26FEF82E291E00E94DC
:100A90005903E4CF0E948B006FEF80E391E00E9446
:100AA0009C012FE78AE196E0215080409040E1F7D9
:100AB00000C0000060E080E391E00E949C0118E12A
:100AC000D9E20FB6F894A895809160008861809370
:100AD0006000109260000FBE6FEF8DE291E00E9407
:100AE0009C0182E291E00E940E04C82F60E08DE23A
:100AF00091E00E949C010FB6F894A89510936000B5
:100B00000FBED0936000A8958C2F90E0FC01319728
:100B1000EC30F105B0F6EE5AFF4F0C94D7050E9469
:100B2000C604CFCF0E94B304CCCF0E94A004C9CF8B
:100B30000E949704C6CF0E948E04C3CF0E947B04FC
:100B4000C0CF0E946804BDCF0E945B04BACF0E9450
:100B50003704B7CF0E942604B4CF0E94D404B1CF8B
:100B600083E391E00E94160142E063E371E080E3D9
:100B700091E00E94550143E063E371E08DE291E072
:100B80000E94550145E063E371E08AE291E00E9432
:100B9000550140E063E371E087E291E00E942402A6
:100BA00041E063E371E084E291E00C942402EE0FF3
:100BB000FF1F0024001C0BBE0790F691E02D099446
:040BC000F894FFCFD7
:100BC40001626F617264696E666F2E680030383A34
:100BD40033303A3434004D617220323920323031AE
:020BE4003900D6
:00000001FF
